:100000004BC065C064C063C062C061C060C05FC0F7
:100010005EC05DC05CC05BC05AC059C058C057C00C
:1000200056C055C054C053C052C051C050C04FC03C
:100030004EC04DC057524F4E470A004F4B212059DA
:100040006F7527726520696E2E205A6865205A6583
:100050006B7269742057657572642049733A0A009F
:10006000456E7465722074686520342D6469676913
:100070007420636F64652E0A0052656164792E0AEC
:100080000045464765666700202B2D2E3031323300
:10009000343536373839680011241FBECFEFD4E02D
:1000A000DEBFCDBF11E0A0E0B1E0E6E8F6E002C0BF
:1000B00005900D92A631B107D9F711E0A6E1B1E0A4
:1000C00001C01D92AC31B107E1F709D0DAC298CF77
:1000D0008091C00087FFFCCF8091C60008952F92C9
:1000E0003F924F925F926F927F928F929F92AF92C8
:1000F000BF92CF92DF92EF92FF920F931F93DF9305
:10010000CF9300D000D000D0CDB7DEB783E390E02E
:100110009FD000D089E790E0EDB7FEB7928381834E
:1001200029D20F900F9050E6252E50E0352E2E014B
:100130000894411C511C45E0642E712C6C0E7D1EF0
:1001400030EDE32E37E0F32E24E3822E20E0922ED2
:100150009BE3A92E90E0B92E8BEBC82E8FEFD82E03
:1001600000D0EDB7FEB73282218204D2F2010F90A7
:100170000F908091C00087FFFCCF8091C600865F02
:100180008193E615F705A9F78981803419F020E0FD
:1001900030E005C0C7010197F1F721E030E08A8126
:1001A0008D3319F020E030E006C02115310519F03B
:1001B000C7010197F1F78B81823419F020E030E01C
:1001C00006C02115310519F0C7010197F1F78C819F
:1001D0008C3329F5232B19F1C7010197F1F700D0D2
:1001E000EDB7FEB7B282A182C5D100E010E00F905A
:1001F0000F90C601801B910BF801E050FF4F20814A
:10020000332727FD3095820F931FD7D10F5F1F4FE4
:100210000730110571F78AE090E0CFD1A1CF00D06F
:10022000EDB7FEB792828182A5D10F900F9098CF43
:100230001F93182F8A3011F48DE0FADF8091C000EF
:1002400085FFFCCF1093C60080E090E01F910895D9
:1002500028E12093C1008093C400892F990F990B46
:100260008093C50088E091E0909319018093180174
:100270000895ABE0B0E0EEE3F1E012C15C014B01A8
:100280007A01FC0117821682838181FD08C06FEF1D
:100290007FEFFEC042E050E0E40EF51E04C03E01D8
:1002A0000894611C711CF501D380F401D3FC859185
:1002B000D3FE81914F01882309F4E7C0853259F4B8
:1002C000D3FC6591D3FE61914F01653219F0062F81
:1002D00010E01AC085E290E029C0002309F4D5C0DF
:1002E00088E890E0602F70E00ED1892B39F403325A
:1002F00011F4106103C00C3661F41068F401D3FCF2
:100300000591D3FE01914F0117FFE7CF002309F4B8
:10031000BCC081E890E0602F70E0F5D0892B49F0F7
:1003200044E050E0E40EF51E8FE390E0B501F6D016
:10033000BACF033629F0033771F00335E1F40AC070
:1003400087010E5F1F4FF70180819181B501E6D0D3
:100350007801A9CF1160F701C080D18003C090E07F
:10036000B501DCD0F60110FD859110FF81916F0180
:100370008823A9F78FCF043611F0093639F517FF16
:1003800008C0F701208131814281538184E090E0EF
:100390000AC0F701808191819C01442737FD409577
:1003A000542F82E090E0E80EF91E1F7E57FF08C030
:1003B00050954095309521953F4F4F4F5F4F1064BA
:1003C000CA01B901A3012AE030E034C00037A9F026
:1003D000013730F40835B1F00F3609F056C006C0C9
:1003E000053739F0083709F050C008C028E030E080
:1003F0000CC01F7E2AE030E008C01061146220E1CA
:1004000030E003C0146020E132E017FF08C0F701BC
:10041000608171818281938144E050E008C0F701DE
:1004200080819181BC0180E090E042E050E0E40EE8
:10043000F51EA301C8D0D82ED618012F10E006FF54
:1004400004C08DE290E0B50169D004FF13C0FE0145
:10045000ED0DF11D8081803369F080E390E0B501FE
:100460005DD002FF07C000721070C801885A9F4F0C
:10047000B50154D0DA94F301ED0DF11D808190E0C7
:10048000B5014CD0DD20B1F70ECFF5016681778143
:10049000CB012B96EEE020C02F923F924F925F92BD
:1004A0006F927F928F929F92AF92BF92CF92DF9284
:1004B000EF92FF920F931F93CF93DF93CDB7DEB7E9
:1004C000CA1BDB0B0FB6F894DEBF0FBECDBF09947D
:1004D0002A88398848885F846E847D848C849B84D4
:1004E000AA84B984C884DF80EE80FD800C811B81E2
:1004F000AA81B981CE0FD11D0FB6F894DEBF0FBE11
:10050000CDBFED010895FC010590061621F00020F5
:10051000D9F7C00108953197CF0108950F931F9324
:10052000CF93DF938C01EB018B8181FF1BC082FF96
:100530000DC02E813F818C819D812817390764F47D
:10054000E881F9810193F983E88306C0E885F9859C
:10055000802F0995892B31F48E819F8101969F838D
:100560008E8302C00FEF1FEFC801DF91CF911F9163
:100570000F910895A0E0B0E0EFEBF2E09DCFFE0117
:10058000359661917191A0911801B091190113965E
:100590008C911397886013968C9380911801909199
:1005A0001901AF0166DEE0911801F0911901238174
:1005B000277F23832096E2E09BCF60911801709102
:1005C0001901ACDF0895FA01AA27283051F1203132
:1005D00081F1E8946F936E7F6E5F7F4F8F4F9F4FD7
:1005E000AF4FB1E03ED0B4E03CD0670F781F891F19
:1005F0009A1FA11D680F791F8A1F911DA11D6A0FE7
:10060000711D811D911DA11D20D009F468943F9199
:100610002AE0269F11243019305D3193DEF6CF0198
:100620000895462F4770405D4193B3E00FD0C9F75E
:10063000F6CF462F4F70405D4A3318F0495D31FDCB
:100640004052419302D0A9F7EACFB4E0A69597951E
:10065000879577956795BA95C9F7009761057105F4
:1006600008959B01AC010A2E06945795479537953E
:100670002795BA95C9F7620F731F841F951FA01D98
:060680000895F894FFCF7D
:10068600B7B5BAADABBFAF00000000020000000076
:0606960018010000000045
:00000001FF
